:1000000012C02CC02BC02AC029C028C027C026C0BF
:1000100025C024C023C069C021C020C01FC01EC08D
:100020001DC01CC01BC011241FBECFE5D4E0DEBF25
:10003000CDBF10E0A0E6B0E0E2E8F4E002C0059039
:100040000D92A036B107D9F711E0A0E6B0E001C0EB
:100050001D92A832B107E1F76FD011C2D1CF0F9333
:100060001F93CF93DF93C0E6D0E008E211E08881D0
:1000700077D0898175D02296C017D107C1F7DF915B
:10008000CF911F910F910895DF92EF92FF920F93FE
:100090001F93CF93DF93C0E6D0E00F2EF8E2EF2E50
:1000A000F1E0FF2EF02D08E310E00F2EF5E1DF2E3A
:1000B000F02DF8018081846080838D2D8A95F1F781
:1000C00080818B7F808380E075D1888380E072D1CE
:1000D00089832296CE15DF0561F7DF91CF911F91BD
:1000E0000F91FF90EF90DF9008951F920F920FB63F
:1000F0000F9211242F933F934F935F936F937F93AE
:100100008F939F93AF93BF93EF93FF938CB18D36F3
:1001100011F4BADFA4DFFF91EF91BF91AF919F91EE
:100120008F917F916F915F914F913F912F910F90A0
:100130000FBE0F901F90189581E090E006D084E2EA
:1001400087BB18BA34D17894FFCFE0E4F0E0908315
:1001500089B982E28BB988E98AB986E880830895F3
:10016000EBE2F0E0908195FFFDCF8CB90895CF933D
:10017000DF93EC018881882329F0F2DF21968881C2
:100180008823D9F7DF91CF910895AF92BF92CF9294
:10019000DF92EF92FF920F931F93DF93CF93CDB730
:1001A000DEB72A970FB6F894DEBF0FBECDBF7B0136
:1001B0008C01611571058105910519F480E3D0DF8B
:1001C00050C0992354F48DE2CBDF10950095F09444
:1001D000E094E11CF11C011D111D6E010894C11C6D
:1001E000D11C0F2EFBE0AF2EBB24F02DAC0EBD1E9C
:1001F000C801B7012AE030E040E050E003D1F60149
:1002000061936F01C801B7012AE030E040E050E09F
:10021000F9D0E22EF32E042F152FCA14DB0441F778
:100220008A85882311F019E00DC019E09E012F5F27
:100230003F4F1150F901E10FF11D80818823C9F36F
:10024000112361F07E010894E11CF11CF701E10F1C
:10025000F11D8081805D84DF1150C1F78981805D4F
:100260007FDF2A960FB6F894DEBF0FBECDBFCF91C9
:10027000DF911F910F91FF90EF90DF90CF90BF9093
:10028000AF900895EF92FF920F931F93DF93CF9358
:1002900000D000D00F92CDB7DEB79C01009719F4C3
:1002A00080E35EDF34C0FE0131968E010A5F1F4F8E
:1002B000C9016AE070E092D08193C9016AE070E000
:1002C0008DD0262F372FE017F10791F78D818823E6
:1002D00011F014E00DC014E09E012F5F3F4F11504C
:1002E000F901E10FF11D80818823C9F3112361F029
:1002F0007E010894E11CF11CF701E10FF11D8081E2
:10030000805D2EDF1150C1F78981805D29DF0F905C
:100310000F900F900F900F90CF91DF911F910F9141
:10032000FF90EF9008950F931F93182F6AE04AD023
:10033000082F48D047D0892F805D12DF802F6AE0D8
:1003400041D0892F805D0CDF812F6AE03BD0892F5F
:10035000805D06DF1F910F910895DF92EF92FF926B
:100360000F931F93CF93DF93C0E0D0E010E8E82E07
:10037000FF24E7FCF09401E30F2EF0E3DF2EF02DD5
:10038000812F90E08E219F21009711F48D2D01C0C7
:10039000802FE6DE16952196C830D10589F7DF91CA
:1003A000CF911F910F91FF90EF90DF9008958CE512
:1003B0008DB908958FB9EEE2F0E080818823ECF7E3
:1003C0008FB10895991B79E004C0991F961708F022
:1003D000961B881F7A95C9F780950895AA1BBB1BA9
:1003E00051E107C0AA1FBB1FA617B70710F0A61B35
:1003F000B70B881F991F5A95A9F780959095BC0156
:10040000CD01089597FB092E05260ED057FD04D087
:1004100014D00AD0001C38F45095409530952195A1
:100420003F4F4F4F5F4F0895F6F790958095709529
:1004300061957F4F8F4F9F4F0895A1E21A2EAA1BFF
:10044000BB1BFD010DC0AA1FBB1FEE1FFF1FA21784
:10045000B307E407F50720F0A21BB30BE40BF50B81
:10046000661F771F881F991F1A9469F7609570950A
:10047000809590959B01AC01BD01CF010895F89442
:02048000FFCFAC
:00000001FF
